:1000000019C028C027C026C025C024C023C022C0D4
:1000100021C020C044C01EC099C02AC01BC01AC045
:1000200019C018C017C016C015C014C013C012C024
:1000300011C010C011241FBECFEFD2E0DEBFCDBF74
:1000400021E0A0E0B1E001C01D92A632B207E1F7C5
:10005000B6D0CAC3D5CF109285001092840081E03B
:100060008093810085E280936F0084E086BB0895D1
:100070001F920F920FB60F9211248F939F9380912E
:100080001F019091200101969093200180931F0100
:100090009F918F910F900FBE0F901F9018951F92F8
:1000A0000F920FB60F9211242F938F939F93AF93BC
:1000B000BF938091000190910101A0910201B09144
:1000C00003010196A11DB11D8093000190930101D0
:1000D000A0930201B093030120912501213061F525
:1000E0008093120190931301A0931401B093150112
:1000F000809186009091870090931C0180931B0152
:1001000080911F019091200190931E0180931D0109
:10011000B09B0FC080911B0190911C0197FD09C0FD
:1001200080911D0190911E01019690931E01809374
:100130001D0182E080932501BF91AF919F918F9126
:100140002F910F900FBE0F901F9018951F920F9236
:100150000FB60F9211248F939F93EF93FF93EAE8CA
:10016000F0E080819181805F984D918380838091C0
:10017000100190911101019690931101809310014B
:10018000FF91EF919F918F910F900FBE0F901F9055
:1001900018959F7090612C9A2B9820E12D9897FFCD
:1001A00002C02A9A01C02A98880F991F2D9A2150BF
:1001B000A9F72B9A2C982C9A2D982A98089580E8C4
:1001C00080936100109261009CE394B991E095B92D
:1001D0008BB984E480BF10922501109216013BDF99
:1001E0007894C1E080916F008B7F80936F00809145
:1001F0001001909111018436910528F0109216019A
:1002000080E090E0C6DF80916F00846080936F0093
:1002100080916F008B7F80936F0080912501811109
:100220000CC08091100190911101892B31F0C09385
:100230002501109211011092100180916F008460CD
:1002400080936F0080912501823061F680911D01BD
:1002500090911E0120911B0130911C01A0E0B0E0A3
:10026000DC0199278827820F931FA11DB11D809360
:10027000170190931801A0931901B0931A0180916E
:10028000170190911801A0911901B0911A014091A4
:100290000401509105016091060170910701841BD2
:1002A000950BA60BB70B8093210190932201A0938D
:1002B0002301B09324018091170190911801A0911E
:1002C0001901B0911A018093040190930501A09344
:1002D0000601B09307018091120190911301A09142
:1002E0001401B091150140910801509109016091EC
:1002F0000A0170910B01841B950BA60BB70B809321
:100300000C0190930D01A0930E01B0930F01809109
:10031000120190911301A0911401B09115018093E5
:10032000080190930901A0930A01B0930B01109268
:10033000250180911601882309F441C060910C01C8
:1003400070910D0180910E0190910F01809021011B
:1003500090902201A0902301B09024012CD120E89C
:1003600036E948E15BE4B9D16B017C01C501B40118
:1003700022D19B01AC01C701B60189D0F62E072F0F
:10038000182FD92F20E036EF4FE157E4A2D11816ED
:1003900024F4F12C06EF1FE1D7E42DEC3CEC4CECFF
:1003A0005DE36F2D702F812F9D2F97D120E030E0DE
:1003B00040E05FE308D0D3D0CB01EBDE13CFC09396
:1003C000160110CF5058BB27AA270ED048C139D1EB
:1003D00030F03ED120F031F49F3F11F41EF42EC1D5
:1003E0000EF4E095E7FB24C1E92F4AD180F3BA1758
:1003F000620773078407950718F071F49EF562C1D0
:100400000EF4E0950B2EBA2FA02D0B01B90190012F
:100410000C01CA01A0011124FF27591B99F0593F73
:1004200050F4503E68F11A16F040A22F232F342FBB
:100430004427585FF3CF469537952795A795F04009
:100440005395C9F77EF41F16BA0B620B730B840B1E
:10045000BAF09150A1F0FF0FBB1F661F771F881FD6
:10046000C2F70EC0BA0F621F731F841F48F487952E
:1004700077956795B795F7959E3F08F0B3CF93951D
:10048000880F08F09927EE0F9795879508950CD05F
:10049000E6C0DED040F0D5D030F021F45F3F19F057
:1004A000C7C0511110C1CAC0EBD098F39923C9F34A
:1004B0005523B1F3951B550BBB27AA27621773076A
:1004C000840738F09F5F5F4F220F331F441FAA1F1E
:1004D000A9F333D00E2E3AF0E0E830D091505040DE
:1004E000E695001CCAF729D0FE2F27D0660F771F8C
:1004F000881FBB1F261737074807AB07B0E809F06E
:10050000BB0B802DBF01FF2793585F4F2AF09E3F02
:10051000510568F08DC0D7C05F3FECF3983EDCF327
:10052000869577956795B795F7959F5FC9F7880F7B
:10053000911D9695879597F90895E1E0660F771FCD
:10054000881FBB1F621773078407BA0720F0621B5E
:10055000730B840BBA0BEE1F88F7E095089598D0C3
:1005600088F09F5790F0B92F9927B751A0F0D1F09C
:10057000660F771F881F991F1AF0BA95C9F712C026
:10058000B13081F09FD0B1E008959CC0672F782FE3
:100590008827B85F39F0B93FCCF386957795679592
:1005A000B395D9F73EF490958095709561957F4FFE
:1005B0008F4F9F4F0895E89409C097FB3EF49095A4
:1005C0008095709561957F4F8F4F9F4F9923A9F02C
:1005D000F92F96E9BB279395F695879577956795BB
:1005E000B795F111F8CFFAF4BB0F11F460FF1BC0FF
:1005F0006F5F7F4F8F4F9F4F16C0882311F096E992
:1006000011C0772321F09EE8872F762F05C066233F
:1006100071F096E8862F70E060E02AF09A95660FF8
:10062000771F881FDAF7880F9695879597F90895B1
:1006300097F99F6780E870E060E008959FEF80EC95
:10064000089500240A941616170618060906089538
:1006500000240A9412161306140605060895092E9E
:100660000394000C11F4882352F0BB0F40F4BF2B0D
:1006700011F460FF04C06F5F7F4F8F4F9F4F08954D
:1006800057FD9058440F551F59F05F3F71F0479543
:10069000880F97FB991F61F09F3F79F08795089528
:1006A000121613061406551FF2CF4695F1DF08C047
:1006B000161617061806991FF1CF86957105610564
:1006C00008940895E894BB2766277727CB0197F90C
:1006D000089566D008F48FEF08950BD0C0CFB1DF36
:1006E00028F0B6DF18F0952309F0A2CFA7CF112488
:1006F000EACFC6DFA0F3959FD1F3950F50E0551FC9
:10070000629FF001729FBB27F00DB11D639FAA2766
:10071000F00DB11DAA1F649F6627B00DA11D661FB5
:10072000829F2227B00DA11D621F739FB00DA11DD6
:10073000621F839FA00D611D221F749F3327A00D90
:10074000611D231F849F600D211D822F762F6A2F2C
:1007500011249F5750408AF0E1F088234AF0EE0FB1
:10076000FF1FBB1F661F771F881F91505040A9F7BE
:100770009E3F510570F05CCFA6CF5F3FECF3983EF3
:10078000DCF3869577956795B795F795E7959F5F25
:10079000C1F7FE2B880F911D9695879597F90895BF
:1007A000990F0008550FAA0BE0E8FEEF1616170682
:1007B000E807F907C0F012161306E407F50798F0EA
:1007C000621B730B840B950B39F40A2661F0232B03
:1007D000242B252B21F408950A2609F4A140A6957F
:0C07E0008FEF811D811D0895F894FFCF5C
:00000001FF
